:020000020000FC
:0200000005C039
:10000A006AC00FED0DBF01E003BF02E009BFBA9A53
:10001A00B898C09AB998C19A789443E06FD013E01F
:10002A0006B3102300000000000006B310230000EE
:10003A000000000006B310231370141749F140FFA3
:10004A0008C010FD06C000E929D00CE327D00FE74D
:10005A0025D040FD08C010FF06C000E81FD00CE301
:10006A001DD00FE71BD041FF08C011FD06C000E9F3
:10007A0015D00DE313D00FE711D041FD08C011FFD1
:10008A0006C000E80BD00DE309D00FE707D0412FD7
:10009A0035D000E800E60FE731D0C1CF2030F1F7C4
:1000AA00302F2AE0089500002843292032303132C7
:1000BA0020576F6C6667616E672044756E637A6558
:1000CA0077736B6900007777772E646D7834796F70
:1000DA00752E646500005FB7203059F02A3021F090
:1000EA00213021F0379510F0C29802C0C29A00C0A0
:1000FA002A950000000000005FBF189500E010E09C
:0A010A001A95F1F70A95E1F7089540
:00000001FF
